:107000006BC00000AAC000008EC000008CC0000051
:107010008AC0000088C0000086C0000084C0000054
:1070200082C0000080C000007EC000007CC0000064
:107030007AC0000078C0000076C0000074C0000074
:1070400072C0000070C000006EC000006CC0000084
:107050006AC0000068C0000066C0000064C0000094
:1070600062C0000060C00000EC2DFD2DB7B6B0FC82
:10707000FDCF27BFE895B7B6B0FCFDCF21E1B7B68D
:10708000B6FCF4CF08950902120001010080320914
:10709000040000000000000012011001FF000008C1
:1070A000C016DC050201010200010E035500530069
:1070B00042006100730070001C03770077007700C6
:1070C0002E00660069007300630068006C002E00EB
:1070D000640065000403090411241FBECFEFD8E04B
:1070E000DEBFCDBF24B7D8E0CEEF39913833399128
:1070F00009F03FEF30933C0120933B0111E0A0E009
:10710000B1E0ECE8F8E702C005900D92A630B107B7
:10711000D9F721E0A6E0B1E001C01D92AB33B20780
:10712000E1F77DD1B1C36CCFA82FB92F80E090E0FB
:1071300041E050EA609530E009C02D918227979593
:10714000879510F084279527305EC8F36F5FA8F30A
:107150000895EADF8D939D930895CF93CFB7CF9392
:10716000DF93C3954C9BE9F74C9B0BC04C9B09C02C
:107170004C9B07C04C9B05C04C9B03C04C9B01C063
:1071800089C06F93C0911E01DD27CB5DDE4F2F9329
:1071900065E54C9B03C02F916F91E6CF0F931F9332
:1071A0004F9320E040E15F9309B1047104FB27F99C
:1071B0003F9350E03BE039C0147140642F77012FBA
:1071C0005F5F1EC0406819B114712F7752501FC005
:1071D000406409B12F770471D1F15F5F00C023C013
:1071E000406219B12F77147191F15F5F00C025C023
:1071F00004711027515012F45D5F00001150279563
:107200002C3F19B1C8F614710127015027952C3F66
:10721000C8F64227499309B1047110274F731150E2
:1072200027952C3FA8F64695469519B1147179F02B
:107230000127015027952C3F98F66B5A60F3315087
:1072400009B1B0F600C011E01CBB002717C03B50CD
:107250003195C31BD04011E01CBB0881033CF9F001
:107260000B34E9F020911C011981110F1213EDCF9D
:10727000093651F10D3211F0013E39F70093230127
:107280003F915F914F911F910F912F916F91CCB3CF
:10729000C0FD67CFDF91CF91CFBFCF9118952091DF
:1072A0002301222369F310912101112339F5343090
:1072B0003AF13093210120931D0110911E013BE012
:1072C000311B30931E011CC0009121010130B4F428
:1072D0000AE53091010134FD14C000930101C1E1C0
:1072E000D1E013C0052710E000C000000BB91AC0A0
:1072F000052710E0221F1DC010E021C04AE502C092
:1073000032ED432FC4E1D0E032E01AB114615C9A4F
:107310000BB11AB954E120E865E320FF05270BB94A
:10732000279517951C3FF0F66695B8F7B1F720FF43
:1073300005270BB9279517951C3FD0F6279517956C
:1073400017FF052700001C3F0BB9B0F629913A95AD
:1073500019F70B7E10912201110FC651D0400BB9C5
:1073600011F010931C0111E01CBB00611AB11B7ECF
:10737000402F4B7E54E05A95F1F70BB91AB94BB92F
:107380007FCFDC0113963C911397932F1496EC91C9
:1073900014978E2F12962C911297203331F4E370AC
:1073A000F0E0EE5FFE4F80810895283529F4311119
:1073B0000EC0E1E0F0E006C0203599F431110CC0B8
:1073C000E0E0F0E089E08093570084910895383040
:1073D00021F5E3E0F0E0F6CF3830F9F4E2E0F0E058
:1073E000F1CF203221F4FC01EE0FFF1F06C028323E
:1073F00031F4FC01EE0FFF1F319684910895203A7D
:1074000009F42CC2203C21F415966C912FD205C0B2
:107410002F3F19F481EF80930F0180E008951AB88F
:1074200080E88BB981E085BF82E085BFE0E0F1E7CD
:10743000A89531978040E1F780913B01877F21F447
:1074400080913C01882371F04F9B0CC0F894549AB2
:107450001BB81DBA1092690081E085BF15BEE0E03F
:10746000F0E009958EEF80930F0114BE0FB6F894EB
:10747000A895809160008861809360001092600000
:107480000FBE80916900826080936900E89A549AE7
:107490008CE0E0E0F5E3A89531978040E1F754985F
:1074A000789410912101135017FD41C180911E0164
:1074B000CCE0D0E0C81BD109CB5DDE4F80911D012F
:1074C0008D3209F0B8C0183009F02FC183EC8093D9
:1074D00011018AE580930101109210013881832FF8
:1074E000807699818823C1F146E051E050932001D4
:1074F00040931F01933031F4CE0143DF80930901A3
:1075000084E08FC0953009F48BC09A3009F488C0AC
:107510008CEF890F8630B0F44A815B8150930E0165
:1075200040930D01993009F491C18E8180930C0133
:107530002D81227020930B0190930A0137FD6CC0BE
:107540008FEF6AC080910F01923011F48E7F01C0DD
:10755000816080930F017AC18A8110921A01911182
:1075600006C010921B012AE131E082E050C0953044
:1075700019F4809322013DC09630A9F59B8191308A
:1075800019F488E990E704C0923041F486E890E766
:107590009093200180931F0182E121C09330F1F488
:1075A000811108C084ED90E79093200180931F0122
:1075B00084E015C0813041F488EB90E7909320017E
:1075C00080931F018CE10BC0823041F48AEA90E77E
:1075D0009093200180931F018EE001C080E090E431
:1075E000909310011EC0983079F0993031F4809357
:1075F00024012AE131E080E00AC081E09A3009F0FC
:1076000080E02AE131E003C024E231E081E0309300
:10761000200120931F0105C090E89093100108C03D
:1076200081E09F81911104C09E81981708F4892FF1
:10763000809300017AC08091100187FF76C000918D
:107640000C01011708F4102F011B00930C01F12C01
:10765000F11608F066C020910A0180910D01909109
:107660000E01273080F06E01FFEFCF1ADF0A68812C
:107670009C012F5F3F4F30930E0120930D01F6D0F8
:10768000F394E601E5CF8115904708F04CC0F394E0
:10769000F394F894E0910D01F0910E012991399144
:1076A00081E0090180935700E89511247894809136
:1076B0000D0190910E01029690930E0180930D01A1
:1076C0008F779927892B51F00111C2CFF11608F459
:1076D000BFCF80910B01882309F4BACFF894E091D1
:1076E0000D01F0910E01329783E080935700E895E9
:1076F000789407B600FCFDCFF894E0910D01F0916D
:107700000E01329785E080935700E895789407B68C
:1077100000FCFDCFF89481E180935700E8957894C0
:1077200097CF011102C010920001109221018091A7
:10773000010184FF67C0809100018F3F09F462C09E
:10774000C82F893008F0C8E08C1B8093000190910D
:10775000110188E8892780931101CC2309F478C0AE
:107760008091100187FF2AC080910C018C1708F4CA
:10777000C82F8C1B80930C01D0900A01D0E082E1CD
:10778000E82E81E0F82ECD1789F100910D011091BE
:107790000E0186E08D1518F4C80160D002C0F80112
:1077A0008491F7018083FFEFEF1AFF0A0F5F1F4FED
:1077B00010930E0100930D01DF5FE5CFE0911F01F3
:1077C000F0912001A2E1B1E086FF07C08C2F9491D7
:1077D0009D9331968150D9F705C08C2F91919D933F
:1077E0008150E1F7F0932001E0931F016C2F82E1BB
:1077F00091E0AFDCCC5FCC3019F08FEF80930001CB
:10780000C093010184E199B1947131F48150D9F7A9
:107810001092220110921C0180910F01803130F0F2
:107820004F9B0FC080910F01805109C04F9909C033
:1078300080910F01823028F080910F018250809357
:107840000F0180910F0181112CCE00CE80E0E9CE96
:1078500060E082E191E07DDCC4E0CFCFF999FECF1A
:1078600092BD81BDF89A992780B50895262FF99980
:10787000FECF1FBA92BD81BD20BD0FB6F894FA9A13
:0C788000F99A0FBE01960895F894FFCF0E
:06788C00FF5A1E950F00DB
:040000030000700089
:00000001FF
